:020000040000FA
:100000003028000000000000F200030E8301F5001C
:100010000A08F4008A010408F300831203138C1EFB
:1000200027281A08981C18281A08181218160D28BC
:1000300083160313F600A10AE3302102031D2228D0
:10004000A230A10021088400760880000D287308E2
:10005000840074088A00750E8300F20E720E090087
:100060008301831603132730810000308C00003099
:100070008D00EF30850000308600B0308700003002
:100080009F0083120313003085000030860000308B
:100090008700C0308B00003090008C0197019D01DB
:1000A000203084008001840A6D300402031C522831
:1000B00002246C24772083160313A230A100A00031
:1000C0008C168312031307142830A4005C30A5009B
:1000D0008F30A6000230A7009220A220C120031C6E
:1000E0006E28A0008F302002031D6E28DB288312AB
:1000F00003130716831603130712143099001815FB
:10010000981683120313181698170712080007127F
:100110008C1E88281A080800871A8C280C1E8E2826
:100120009900080007100130A900B4200030A90090
:10013000B4200030A900B420A730A900B42087154E
:10014000871108000430A900B4202708A900B420B2
:100150002608A900B4202508A900B4202408A90075
:10016000B4208715871108000830A1000310A90DDD
:1001700003180715031C071187148710A10BB72854
:100180000800831603132108200283120313031DA2
:10019000CB280310080083160313A00AE3302002C3
:1001A000031DD428A230A000200884000008831278
:1001B0000313031408008021C120031CDC28E8007D
:1001C00060306802031880214F3084004E08840795
:1001D00068088000CE0A4F08773A031DF6284E08BB
:1001E000163A031DF6282A1486227E294F08663AFD
:1001F000031D00294E080A3A031D0029B2237E2957
:100200004F08783A031D0B294E08163A031D0B2997
:100210002A1086227E294F086D3A031D15294E08A3
:10022000013A031D15297C237E294F08653A031DD9
:100230001F294E080D3A031D1F29C2237E294F088E
:10024000763A031D29294E08013A031D2929FE2368
:100250007E294F08723A031D33294E08023A031DC6
:10026000332908247E294F08613A031D3E294E0890
:10027000193A031D3E292A1084227E294F08623A2A
:10028000031D49294E08193A031D49292A148422BD
:100290007E294F08733A031D53294E08013A031D66
:1002A0005329EE237E294F086F3A031D5D294E081E
:1002B000023A031D5D2901247E294F08633A031D7C
:1002C00068294E081B3A031D68292A10DE227E2960
:1002D0004F08643A031D73294E081B3A031D732906
:1002E0002A14DE227E294F086E3A031D7D294E080E
:1002F000013A031D7D298D237E29DC2880216E286B
:100300000A220800D201D301D401D501D601D701B8
:10031000CE01CF01D001D10108008221480884001C
:100320000008CE00840A0008CF00840A0008D0002C
:10033000840A0008D100840A0008D2002830AB00EB
:100340000310D20CD10CD00CCF0CCE0CD70CD60C89
:10035000D50CD40CD30C4E3084000530AC00801F7B
:10036000B32930308002801DB72903308002840A0F
:10037000AC0BAF29AB0BA0294808840053088000C0
:10038000840A54088000840A55088000840A5608AC
:100390008000840A5708800008002E08D8002F0823
:1003A000D9003008DA003108DB003208DC002030E8
:1003B000D6005830C8006030C900CF010310D50CFA
:1003C000D40CD30CD20C031CFE290830D0004808F2
:1003D00084000008CE00490884004F08CF01800740
:1003E000031CF4290130CF004E088007031CFA29B2
:1003F0000130CF00C80AC90AD00BE7290310D80D75
:10040000D90DDA0DDB0DDC0DDD0DDE0DDF0DD60BAC
:10041000D92908004E308400800167300402031996
:10042000132A840A0C2A080050080F39B800510E0C
:10043000F039B70052080F39B704530EF039B6003F
:1004400054080F39B604550EF039B50056080F3967
:10045000B504570EF039B40058080F39B404080039
:10046000BD01590EF039BC005A080F39BC045B0EAF
:10047000F039BB005C080F39BB045D0EF039BA00DF
:100480005E080F39BA045F0EF039B90060080F3901
:10049000B9040800C001C101C201610EF039BF00FA
:1004A00062080F39BF04630EF039BE0064080F39CB
:1004B000BE040800C401C501C601C70165080F39A3
:1004C000C404660EF039C30067080F39C30408007E
:1004D000FB01FC01FD01FE01FF01680EF039FB008C
:1004E00069080F39FB0408004308EA004408EB00E0
:1004F0000F30E900E90B7A2AEA0B782AEB08031996
:10050000832AEB03782A08005A22882AC301C401EF
:100510008316031380309F008312031314223022AA
:100520004A223430C8008D213930C8008D213E3038
:10053000C8008D214330C8008D210A223508D30020
:100540003408D2003608D4003708D500CD21202445
:10055000C308031DAF2AC408031DAF2AB02A7422A2
:100560002D2422088E2023088E202B2422088E2062
:1005700023088E203908B4073A0803183A0FB50744
:100580003B0803183B0FB6073C0803183C0FB7079E
:100590000A223508D3003408D2003608D4003708C0
:1005A000D500CD212024BE033E0A0319BF03BE0897
:1005B000031DA82ABF08031DA82A080083160313D9
:1005C00080309F008312031368225A2214223022A3
:1005D0004A223430C8008D213930C8008D213E3088
:1005E000C8008D214330C8008D217B30C8008D218B
:1005F0000A223508D3003408D2003608D400370860
:10060000D500CD21202487246E237808FA007708AE
:10061000F9007808E7007708E6008F243230C00040
:10062000E001C0080319162BC0038B244408D9002D
:100630004308D800A2246E237808E3007708E2007C
:100640007808E7007708E6007908E2027A08031CD8
:100650007A0FE302E31F312BE209E309E20A0319EF
:10066000E30A63087C0203183E2BE00A0530C00051
:100670008F246708FA006608F9001B2B6708FA0048
:100680006608F90060088E2000308E2066088E20F3
:1006900067088E203908B4073A0803183A0FB507DF
:1006A0003B0803183B0FB6073C0803183C0FB7077D
:1006B0000A223508D3003408D2003608D40037089F
:1006C000D500CD212024BE033E0A0319BF03BE0876
:1006D000031D102BBF08031D102B08002030AB009A
:1006E000F701F8012B242208F70723080318230F2A
:1006F000F807AB0B722B08008316031380309F00A2
:10070000831203132F2422088E2023088E202B24EB
:1007100022088E2023088E200800831603138030C1
:100720009F0083120313F701F801F901FA01203049
:10073000AB002F242208F70723080318230FF8071C
:100740002B242208F90723080318230FFA07AB0B01
:10075000992B77088E2078088E2079088E207A08C9
:100760008E20080014223430C8008D210A2235085A
:10077000D3003408D2003608D4003708D500CD2184
:100780002024080050081824B200B20E5108182482
:10079000B20452081824B100B10E53081824B10451
:1007A00054081824B000B00E55081824B004560898
:1007B0001824AF00AF0E57081824AF0458081824A7
:1007C000AE00AE0E59081824AE045A081824B3001F
:1007D000B30E5B081824B3047924302802308E202D
:1007E0006C088E208316031380309F00831203133E
:1007F000292422088E2023088E20080078308E209D
:100800000800080086013F308600B12486010800F8
:100810005008EC0086016C188614EC1806156C194B
:100820008615EC1906166C1A8616EC1A06170800BF
:10083000CE0041304E023030031837304E020800EF
:100840006508A5006408A4006608A6006708A7005C
:10085000A2289130322CA130322C2A18312C893028
:10086000322C81309F0040241F151F19352C831610
:1008700003131E0883120313A2001E08A30008001E
:10088000C830CE00CE0B422C0800831603178C18FC
:10089000472C8312031770088D0071088C00831693
:1008A00003178C130C158B1355308D00AA308D0057
:1008B0008C148B170C118312031308008312031777
:1008C00070088D00831603178C130C148312031702
:1008D0000C088312031308000630AB002E3084008E
:1008E0000030F0005E248000840AF00AAB0B722C0A
:1008F00008000630AB000030F0002E308400000805
:10090000F1004524840AF00AAB0B7F2C0800FA3072
:100910009624FA309624FA309624FA30962C6430D5
:10092000962C0A30962C0530962C0130EB000730BF
:10093000EA007C30E900E90B9B2CEA0B9B2CEB0BCB
:10094000972C0800D808031DA82CD9080319B02C2F
:100950009524D803580A0319D9030319D808A22CDF
:1009600008001A30EB007730EA005530E900E90B57
:0E097000B72CEA0BB72CEB0BB72C08000000DD
:02400E00723FFF
:0C42000018007100C700BC000A0000009C
:00000001FF
